:03000000024EFBB2
:0C4EFB00787FE4F6D8FD7581A3023889A9
:0D001600E4F576752CF3A82CE2F576FF22B8
:104E1200752CF3A82CE2F562752CF4A82CE25562ED
:044E2200F576FF2200
:104DD300752CF3A82CE2F562752CF4A82CE255622D
:054DE300F5766FF222DD
:104E2600752CF3A82CE2F562752CF4A82CE25562D9
:044E3600F576F222F9
:104B2700E54524FE600F146011146013240370140C
:104B3700751004801275100C800D7510148008759F
:0E4B4700101C80037F0022E4FDAF10124A60B4
:014B5500223D
:10438D008F0F752CF6A82CE254F0F50F1206ED43A5
:10439D00E42043DF3043DA4043DA5043DA6043DA56
:1043AD007043CA8043CA9043CAA043CAB043CAC02F
:1043BD0043CAD043CAE043CAF0000043E9124B2779
:1043CD00BF5905750FFF8017750F808012750F404F
:1043DD00800D750F108008750F208003750F80AF4D
:0243ED000F229D
:0E4EB600755F3C752CF4A82CE25FF576F222B5
:104E4E00755F03752CF4A82CE25480F576F2E55FBD
:034E5E0070FC22C3
:104DA700752CF4A82CE25FF576F2A82CE25FF57675
:064DB7006F60F77F01228E
:104D5B00752CF4A82CE25FF5766F6002EFF2A82CAD
:0A4D6B00E25FF576B507F77F01223D
:024BFD008F081F
:104BFF00AF4512438D8F09E50964406008752CF4A9
:104C0F00A82CE508F2AF4512438D8F09E509B44092
:034C1F00F47F011E
:014C2200226F
:02498100AD0780
:10498300E54524FE600F14601114601324037014B2
:10499300750804801275080C800D7508148008755D
:1049A300081C80037F0022E4FBAF08124B82BF0187
:0649B300037F01227F00DA
:0149B90022DB
:023A22008F0A09
:103A2400E4F50B7B6A7D807F52123B7AEF7002FFD4
:103A3400227B6C7D807F50123B7AEF7002FF22E480
:103A4400F50B124E12EF650A6007AF0A124DD380D0
:103A5400067567307F0122756E7D124E12EFB50A2E
:103A640006756E01750B01E56ED3940150ECE50B00
:103A7400B4010AE565B452057F0F124ED9E56564B9
:103A8400507029E50A6025756EFFAF4512438DBF5E
:103A94004003756E01E56ED3940150EEAF451243B9
:103AA4008DEF6440600675674B7F0022E50BB4011F
:103AB400067567307F0122E565B4520575674A8053
:063AC4000375674B7F0053
:013ACA0022D9
:103C14008F0EE50EB42003750E08ED24FE6030040B
:103C2400705AE50E2482FF7512107B10E4FD124DCC
:103C3400E8E50E2484FF7512067B10E4FD124DE8BE
:103C4400E50E2486FF7512107B2EE4FD024DE8E597
:103C54000E2482FF7512107B11E4FD124DE8E50E6F
:103C64002484FF7512067B10E4FD124DE8E50E2452
:103C740086FF7512117B2EE4FD024DE8E50E2482C9
:103C8400FF7512117B10E4FD124DE8E50E2484FF4C
:103C94007512067B11E4FD124DE8E50E2486FF75CE
:0A3CA40012107B2EE4FD124DE82201
:103EE2007F01124ED9752CF2A82C74FFF2755D3247
:103EF200E4F512FBFD7F03124DE8C3E5409533E57F
:103F02003F953250177D027F02124A608F317D0247
:103F12007F03124A608F5EE4F56080157D027F02A6
:103F2200124A608F317D027F03124A608F5E756094
:103F3200017D01E4FF123C14855E12AB31E4FD7F8A
:103F420006124DE8AB4BAA4CA94D12044EFBC0031E
:103F5200AB4B900001120467F512D003E4FDFF029F
:023F62004DE828
:1031F0008F0D756003E4F512FBFD7F06124DE8E5C7
:103200000D24B270030232D424FA605424FD7003FA
:1032100002329024F6601624F370030232CF24FAAF
:10322000603624FD6065243660030232E7E4F5125F
:10323000FBFD7F03124DE8AB46AA47A94812044E96
:10324000FBC003AB46900001120467F512D003E403
:10325000FDFF124DE80232E7E56C30E0030232E791
:10326000E4F512FBFD7F01124DE8AB46AA47A948E1
:1032700012044EFBC003AB46900001120467F51226
:10328000D003E4FD7F02124DE8805CE56C20E0573E
:10329000AB4BAA4CA94D12044EFBC003AB4B9000A4
:1032A00001120467F512D003E4FD7F02124DE8AB72
:1032B0004BAA4CA94D12044EFBC003AB4B9000012E
:1032C000120467F512D003E4FDFF124DE88018E503
:1032D0006C20E013E4F512FBFDFF124DE8E4F5125B
:1032E000FBFD7F02124DE87566FF7D02E4FF023CA4
:0132F00014C9
:103D48007F03124ED9752CF2A82C74FFF2755032ED
:103D5800E4F512FBFD7F23124DE8C3E5409533E5FA
:103D68003F95325005E4F5568003755601752CF1E0
:103D7800A82CE25408F576B4080DE565B44F08752B
:103D88003102755EFF80127D027F22124A608F31F8
:103D98007D027F23124A608F5E7D017F20123C14D2
:103DA800855E12AB31E4FD7F26124DE8AB4BAA4C81
:103DB800A94D12044EFBC003AB4B900001120467DF
:0B3DC800F512D003E4FD7F20024DE85F
:102B78008F0D755603E4F512FBFD7F26124DE8E52F
:102B88000D24BF603024F37003022C6624FA6059C8
:102B980024FD7003022C2124E97003022C6124FA1D
:102BA800603F24FD606E24166003022C7AE56C30C9
:102BB800E203022C7AE4F512FBFD7F23124DE8AB09
:102BC80046AA47A94812044EFBC003AB4690000131
:102BD800120467F512D003E4FD7F20124DE8022CA1
:102BE8007AE56C30E203022C7AE4F512FBFD7F21D2
:102BF800124DE8AB46AA47A94812044EFBC003ABE6
:102C080046900001120467F512D003E4FD7F2212FA
:102C18004DE8805EE56C20E259AB4BAA4CA94D12F9
:102C2800044EFBC003AB4B900001120467F512D0B1
:102C380003E4FD7F22124DE8AB4BAA4CA94D1204C8
:102C48004EFBC003AB4B900001120467F512D00392
:102C5800E4FD7F20124DE88019E56C20E214E4F5CC
:102C680012FBFD7F20124DE8E4F512FBFD7F2212D6
:102C78004DE87566FF752CF1A82CE25408F576B47A
:102C8800080B7D027F20123C14757208227550FFD4
:042C9800E4F57222CB
:1037A9008F0CE50CB46305750C4380287F611231D9
:1037B900F07B617D7D7F56123B7AEF70177F611236
:1037C90031F0E567B44203756730E4F58E789E768B
:1037D90030758E027F611231F0E50C64437025F576
:1037E90012FBFD7F06124DE8752CF1A82CE254045A
:1037F900F576B4040AE4F512FBFD7F02124DE8E404
:10380900F53FF540123EE2E50C644A60707B627D4B
:103819007D7F56123B7AEF7014E560700575673647
:1038290080037567377F611231F07F00227F611253
:1038390031F0E50C64437040752CF1A82CE2540476
:10384900F5767034F512FBFD7F06124DE87512FF0F
:103859007BFFE4FD7F02124DE8E4F53FF540123E9F
:10386900E27B627D7D7F56123B7AEF700B7567367E
:103879007F611231F07F0022AF0C1231F07F0122FB
:10483600752CF1A82CE25404F576702FF512FBFDC9
:104846007F06124DE87512FF7BFFE4FD7F02124DD5
:10485600E8E55CB40305750B638003750B43AF0B8A
:104866001237A9EF700B756736FF22E4FDFF123C85
:03487600147F01AB
:01487900221C
:104450008F0CE50CB46305750C6180237B617D7D59
:104460007F48123B7AEF70177F61122B78E567B4B3
:104470004203756730E4F58E789E7630758E0212B1
:104480003D48E50C644A60257B627D7D7F48123B98
:104490007AEF7014E55670057567358003756735DA
:1044A0007F61122B787F0022AF0C122B787F0122C4
:102C9C00750B01752CF1A82CE2FF5408F5767066C3
:102CAC00EF5410F5767023F512FBFD7F26124DE8DC
:102CBC007512407B9CE4FD7F22124DE8753F4E75EA
:102CCC004020E4F55C7F63124450752CF1A82CE293
:102CDC00FF5408F576702CEF5410F57664107023C1
:102CEC00F512FBFD7F26124DE87512207B4EE4FD9C
:102CFC007F22124DE8753F79754018E4F55C7F61D1
:102D0C00124450755C02752CF1A82CE25408F5762F
:102D1C006408707B7F01124ED9E4F512FBFD7F260F
:102D2C00124DE87512F87B75E4FD7F22124DE875A3
:102D3C003F717540487F63124450EF7004F50B806F
:102D4C00517F01124ED9753F797540187F6112443D
:102D5C0050EF7004F50B803A7F01124ED930001001
:102D6C007B007A00793FE4F5107F061244B0800EA8
:102D7C007B007A00793FE4F5107F6E1244B07F61DE
:102D8C00124450EF7004F50B8008750B018003E4BE
:102D9C00F50B7F61122B78752CF1A82CE25408F5F9
:072DAC00767002F50BAF0B7E
:012DB30022FD
:1047A8008F0B7F431237A9EF7002FF22856A3F857E
:1047B8006B407F61124450EF7002FF22E565B452EE
:1047C80010E50B7005754FF5800CAF0B12000380D8
:1047D80005AF0B12000385703F8571407F6112376A
:0947E800A9EF7002FF227F0122FB
:10490000E4F568F561F57375270BF575756730D2B9
:1049100017F54B754C00754D3FF5467547007548CA
:1049200032F529752A00752B77F58E789FF6087673
:10493000000876A2758E02F56AF56B755AFFD214DF
:014940002254
:10432400C296D296C295D295C294C294C293D293A5
:10433400D2A3D2A4D2A6C2A7C2A7C2A5C2A5C2A212
:10434400D2A2C2A1D2A1C2A0D2A0C2B5D2B5D2B4C7
:10435400758E02C2A8D28AD2AAC2AED2AFD2BAE4B1
:10436400FF7F0B7834745FF608DFFCE4F58EFFE41E
:10437400FEEF75F00CA424002EF8745FF20EBE0C50
:08438400F00FBF0CEA758E0278
:01438C00220E
:104E3A00759850438780C2CAD2CCD2CD75CBFFD2E7
:044E4A00CAD2AC22FA
:104E86005389F0438901E4F58CF58AD28CD2A922A4
:0100110022CC
:1043EF00E4FD7FF9124A608F28E528C3947F500CB3
:1043FF0075287FE4FBAD287FF9124B828528CAE42C
:10440F00F58E789E763074FF7890F208F27894E407
:10441F00F20874FFF27896E4F20874FFF27898E4E9
:10442F00F20874FFF2789AE4F20874FFF2789CE4D1
:10443F00F20874FFF2758E02C211C212F55DF550CB
:01444F00224A
:10396900E4F521F520F5621200168F62752CF0A896
:103979002CE25403F57624FE700875590253628FC0
:1039890080037F0022E5625480FF700585622180F3
:1039990057E5625470FF24F0601C24F0601824F08D
:1039A900601424F0601A24F0601624F0601E24F0DC
:1039B900602824707032E562543FF521D2008028D6
:1039C900E562541FF521D200D201801CE562540F33
:1039D900F521D200D201D206800EE562540FF521FD
:1039E900D200D201D206D207752CF0A82CE2FF54DE
:1039F90001F576B40102D202EF5402F576B402025F
:103A0900D203EF5404F576B40402D204EF5408F556
:083A190076B40802D2057F011A
:013A21002282
:1035D900E4FD7FFF124A60EF645A605FE4FD7FFFFC
:1035E900124A60EF647A6003124C6D1248BDE4FB25
:1035F9007D5A7FFF124B82EF7002FF22123969EF69
:103609007002FF22E4FBAD207FFC124B82EF7002B7
:10361900FF22E4FBAD217FFD124B82EF7002FF22F6
:10362900E4FBAD597FFE124B82EF7002FF22124676
:1036390070752CF7A82C7402F2807A123969EF7030
:1036490005755A28FF22E4FD7FFE124A608F5AE56C
:103659005AB42E11755A28E4FBAD597FFE124B82DC
:10366900EF700EFF22E55A65596006755A287F00EA
:1036790022755A28E55924FE703B300011E4F55AA9
:10368900300B03755A50300A1D755A508018300B8B
:1036990003E4F55A300A03E4F55A300903E4F55A0C
:1036A900300803E4F55A752CF3A82CE25470F5762A
:0F36B9006003755A3CE55A70037F01227F00229F
:10450F00124B561232F1121DC1752CF0756E78E5F3
:10451F006E24EC603724EC602C24EC602124EC60DA
:10452F001624EC600B24EC7028A82C7403F2802165
:10453F00A82C7402F2801AA82C7403F28013A82CF2
:10454F007402F2800CA82C7403F28005A82C74025C
:0C455F00F2E56E70BAA82CF21242B922EC
:10388900124900124324752CF0A82C7402F2124E2E
:103899003A124E861200111243EF755C031235D9A4
:1038A900BF011C7F2D124ED912450FBF010C752C7B
:1038B900F0A82C7401F2F55C800D755C0280087526
:1038C9002CF0A82C7403F2D2A9D2AA120D67752C78
:1038D900F0E55CB40107A82C7401F28048E5637037
:1038E90005855A63803FE56324E2603524F6602A42
:1038F90024F6602024F6601524F6600B24F6702562
:10390900A82CE55CF2801EA82CE4F28018A82CE50E
:103919005CF28011A82CE4F2800BA82CE55CF28003
:1039290004A82CE4F2E55D64016004E5667010E426
:10393900F55DFDFF123C147560037F01120003E57C
:103949005064016007E56660030238D0E4F550FD74
:103959007F20123C147556037F011200030238D0F0
:03000B000240DED2
:1040DE00C0E0C0D0E564B401057564008069756404
:1040EE0001E56E6002156EE56660021566E55F60BD
:1040FE0002155FE55860021558E55B6002155BE539
:10410E006360021563E54F6026C394C85015154FC2
:10411E00301405754F00D2A2E54FB40118D2A2D2C9
:10412E00148012054FE54F700CC2A2C214800620F7
:10413E00A203754F2DE55DD394014002155DE55048
:0C414E00D3940140021550D0D0D0E032D4
:030023000246C0D2
:1046C000C0E0C0D075D000C000C007309831C2989B
:1046D00074342568F8E6645F7025755B14A69974D8
:1046E000342568F8E6FF645A6013EF647A600EE5DB
:1046F00068B40A05756800800605688002765F3038
:0F4700009904C299D217D007D000D0D0D0E032A0
:030013000218AC24
:1018AC00C0E0C0F0C083C082C0D075D000C000C002
:0D18BC0001C002C003C004C005C006C00783
:1018C900858E16758E02752CF2A82CE2F5765410C9
:1018D900F562641070497410F2751A00E4FBFD7F1B
:1018E9002A12424D751A037B03E4FD7F3412424DDF
:1018F900751A00E4FBFD7F2612424D751A207B4EB6
:10190900E4FD7F2012424D751A207B4EE4FD7F22B3
:1019190012424D751A007B03E4FD7F3412424DE5F6
:10192900765408F56264086003021A0AA82C740840
:10193900F2E556B40302D213E55664017072E55C10
:101949007049755C02F51AFBFD7F2A12424D751A22
:10195900037B03E4FD7F3412424D751A00E4FBFD5D
:101969007F2612424D751A307B75E4FD7F201242A5
:101979004D751A307B75E4FD7F2212424D751A00B0
:101989007B03E4FD7F3412424D8076751A00E4FB37
:10199900FD7F2612424D751A307B75E4FD7F2212B8
:1019A900424D855E1AAB31E4FD7F2612424D8051CE
:1019B900E55C6401604BE55C7047755C02F51AFBF8
:1019C900FD7F2A12424D751A037B03E4FD7F341211
:1019D900424D751A00E4FBFD7F2612424D751AF837
:1019E9007B75E4FD7F2012424D751AF87B75E4FD85
:1019F9007F2212424D751A007B03E4FD7F341242A7
:101A09004DE5765404F5626404704AA82C7404F216
:101A1900E5607041F51AFBFD7F0A12424D751A0304
:101A29007B03E4FD7F1412424D751A00E4FBFD7F30
:101A39000612424D751A00E4FBFDFF12424D751A5C
:101A490000E4FBFD7F0212424D751A007B03E4FDA1
:101A59007F1412424DE5765402F56264027068A85B
:101A69002C7402F2E56064016003021B2B756002AD
:101A7900F51AFBFD7F0A12424D751A037B03E4FD3B
:101A89007F1412424D751A00E4FBFD7F0612424D88
:101A9900751A00E4FBFD7F0312424DAB46AA47A924
:101AA9004812044EFBC003AB46900001120467F5CF
:101AB9001AD003E4FDFF12424D751A007B03E4FDC1
:101AC9007F1412424D805BE5765401F56264017022
:101AD90051A82C04F230154A6560704620164375EA
:101AE9006002751A607B01FD7F0A12424D751A006A
:101AF900E4FBFD7F0312424D74EE2578F5787402FC
:101B09003577F577AB29AA2AA92B12044EFBC00316
:101B1900AB29900001120467F51AD003E4FDFF1206
:051B2900424D85168EFF
:101B2E00D007D006D005D004D003D002D001D0000B
:0B1B3E00D0D0D082D083D0F0D0E032B5
:1034E5005400424450004447485056004450534D00
:1034F5005400414856004F005352005300554400B4
:10350500434F5354004447505259004400414347E8
:10351500494F515253565700434F00424344474D7C
:103525005052535400435253004C534B2D44617435
:1035350061003639383731005000414749004D00A8
:103545004344454C53545600424856000A0D004327
:10355500005200425245544D00525700424957000F
:103565004200446973634A657420342020566572AD
:103575002E20332E34730053687574746C652020C7
:1035850020205665722E20352E3067004F75743A0F
:10359500200020496E3A2000202020005649203D79
:1035A50020005658203D20005641203D2000565011
:1035B500203D20004849203D20004858203D20005E
:1035C5004841203D20004850203D200056480041FC
:0435D5004950580001
:104061008F09E4F58EFB7D08AF0912470F7892E6C0
:10407100FF789F860308E6FA08E6F9EF12049478C0
:1040810093E6FF789F860308E6FA08E6F9900001B7
:10409100EF1204A678A2E6F57008E6F5717894E6C9
:1040A100F56508E6F56D08E6F56F08E6F54E08E6F4
:1040B10012049408E6FF789F860308E6FA08E6F9F9
:1040C100900001EF1204A678A2E6F56A08E6F56B06
:0D40D10085284A857445850941758E0222B7
:1030E500756730BF0108855128854374800685536F
:1030F50028854474E52824FE602C1470030231A74A
:103105001470030231B81470030231D12404600332
:103115000231E2E5741470087F801240610231E5E6
:103125007567330231E5E574146028146035146061
:103135004114604D246B605824997061752804759D
:103145007401300008E4FF1240610231E575673310
:103155000231E53008087F201240610231E57567CC
:1031650033807D3009077F2812406180737567338E
:10317500806E300A077F3012406180647567338046
:103185005F300B077F38124061805575673380507B
:103195007528057574017F68124061804375673332
:1031A500803EE5741470077F701240618032756748
:1031B50033802DE57414700F300007E4FF12406171
:1031C500801E75673380197567338014E574147034
:1031D500077F681240618008756733800375673320
:0B31E500E567B430037F01227F002269
:104C8F007F01123FE3EF7004FF024DBD7F01123031
:0F4C9F00E5EF7004FF024DBD1215F6124DBD2258
:104CAE007F01123FE3EF7004FF024DBD7F01123012
:0F4CBE00E5EF7004FF024DBD122430124DBD22F0
:1049F200752CF1A82CE25401F576B4011C75510511
:104A02007543017F011230E5EF7004FF124DBD12B4
:104A12002430EF7004FF124DBDE565B4590375658E
:074A2200521242B9024DBD22
:103ACB007BFF7A3479E5124949EF24AC6003023B62
:103ADB005F7BFF7A3479E7124949EF24BC604224BB
:103AEB00F46009240E70687F01024DBD755103759A
:103AFB0043017F011230E5EF7004FF024DBD7F43A0
:103B0B001237A9EF7007756736FF024DBD124C498E
:103B1B00EF7004FF024DBD7F011247A87F01024DDC
:103B2B00BD7F01123FE3EF7004FF024DBD7F011219
:103B3B0030E5EF7004FF024DBD7F431237A9EF70E4
:103B4B0007756736FF024DBDE4FF1247A8800A7F59
:103B5B003F024DBD7F3F024DBD7F011230E5EF644B
:093B6B00016005E4FF124DBD22CA
:101B4900E52704FDE4FF1247F17BFF7A3479EB12B4
:101B59004949EF24B97003021BF9147003021C7779
:101B690024F87003021CB124FA7003021D812412A7
:101B79006003021DBB7BFF7A3479F1124949EF24D6
:101B8900BC7003021DC024F7603E24FA603414605F
:101B99003D240470567BFF7A3479F7124949EF24C2
:101BA900B8600E24F2601024157012124670024DAE
:101BB900BD12000E024DBD122ECA024DBD7F3F025D
:101BC9004DBD124C23024DBD1233F0024DBD7F01B4
:101BD900124DBD1248BDE4FB7D7A7FFF124B827521
:101BE9008E02752CF7A82C7402F2227F3F024DBD9C
:101BF9007BFF7A3479FB124949EF24B1706B7BFF83
:101C09007A3479FD124949EF24AE603214705512C5
:101C19003E5BE574B4FF05E4FF024DBDE574D39462
:101C2900134003757413E57475F00CA4240AF57454
:101C3900E4FBAD747FBC124B827F01024DBDE4FD14
:101C49007FBC124A608F74E574B40A06E4FFFE0291
:101C59002FD874F62574F57475F00C84F574FF7E2D
:101C690000022FD87F3F024DBD7F3F024DBD7BFF54
:101C79007A357900124949EF24AD70277BFF7A350F
:101C89007902124949EF24BC600C24EF70107FFFE0
:101C9900123F64024DBD7F01123F64024DBD7F3F7B
:101CA900024DBD7F3F024DBD7F01123FE3EF70033F
:101CB900021D7C7F011230E5EF64016003021D7C87
:101CC900E55C64016003021D72E56764366005E541
:101CD90067B4370FE55CB4010A1242B9EF7004FF2B
:101CE900124DBD7B6C7D807F52123B7AEF70077578
:101CF900674BFF024DBDE56524AE60232402705B8E
:101D0900756EFF7F0112438DEF5480F562B4800434
:101D1900E56E70EFE56E700775674BFF024DBDE428
:101D2900F5080508AF6D123A22BF01037508F0E501
:101D390008C3940440ECE50864F06017E56524B035
:101D4900600924FE700875674A800375674BE4FFD4
:101D5900024DBD7F19124ED975690175673012257B
:101D6900EFBF010F7F01024DBD756738AD677F3841
:101D7900124CEBE4FF024DBD7BFF7A357900124925
:101D890049EF24AD70277BFF7A357902124949EF73
:101D990024BC600C24EF70107FFF12415A024DBD24
:101DA9007F0112415A024DBD7F3F024DBD7F3F0267
:071DB9004DBD7F3F124DBD3F
:011DC0002200
:104A29007F01123FE3EF7004FF024DBD7F02123F89
:104A3900E3EF7004FF024DBD7F011230E5EF700412
:104A4900FF024DBD7F021230E5EF7004FF024DBD3C
:074A5900124BD6124DBD22E5
:102DB400E52704FDE4FF1247F17BFF7A357905121C
:102DC40049498F62E562B4540B7BFF7A35790A1264
:102DD40049498F627F01123FE3EF7003022EC47FE3
:102DE400011230E5EF64016003022EC4E56564500E
:102DF4006003022EC4E56224BC7003022EA124FDEC
:102E04007003022EA924F86023147003022EAF2449
:102E1400FE7003022EB714601B24FA607824166037
:102E240003022EBFAF6D124DA7024DBDAF6D124B05
:102E3400FD024DBD756EFAAF4512438DBF8004E5AA
:102E44006E70F4AF4512438DEF24F0603024F060CF
:102E54002024E0601024C070307F42124D81AD67A1
:102E64007F42024CEB7F4F124D81AD677F4F024C86
:102E7400EB7F49124D81AD677F49024CEB7F4312D2
:102E84004D81AD677F43024CEB7F45124D81AD67A9
:102E94007F45024CEB7F59124981024DBD7F44129C
:102EA4004981024DBD124B27024DBD7F501249810D
:102EB400024DBD7F52124981024DBD7F3F024DBD7F
:052EC400E4FF124DBD0A
:012EC90022E6
:1049BA00E52704FDE4FF1247F17BFF7A35791012EF
:1049CA004949EF24BC701B7BFF7A35791212494999
:1049DA00EF24AF7008756748E4FF024DBD7F3F02C0
:0849EA004DBD7F3F124DBD22BF
:0E4EC400E52704FDE4FF1247F1AF67024DBD84
:10461F00E52704FDE4FF1247F17BFF7A35791D1280
:10462F0049498F627F01123FE3EF602F7F01123004
:10463F00E5EF64017025E5656452701FE56224B1F2
:10464F00600C240C7010AF6D124DA7024DBDAF6DF5
:10465F00124D5B024DBD7F3F024DBDE4FF124DBDBC
:01466F002228
:10071300E52704FDE4FF1247F17BFF7A35792012C8
:100723004949EF24BD7003020B0C24FC700302083B
:10073300AE24FA7003020B2024FD70030208182470
:10074300FE7003020C86147003020D24147003025E
:10075300085524126003020D617BFF7A35792A1252
:100763004949EF24AE601314604D2410600302085E
:10077300137BFF7A35792E024A94E4FD7FF9124AFE
:10078300608F28E5282481602424C0601B24E06056
:100793001224F5600924F570197F31024DBD7F37AE
:1007A300024DBD7F38024DBD7F39024DBD7F3602FC
:1007B3004DBD7F3F024DBDE4F5287BFF7A35793788
:1007C300124949EF24CF602624FA601B14601114E8
:1007D30060072403703575287FE52870037528BFEB
:1007E300E52870037528DFE52870037528EAE528F6
:1007F30070037528F5E528600DE4FBAD287FF91239
:100803004B828528CA22E4FF024DBD7F3F024DBDC6
:100813007F3F024DBD7BFF7A35793D124949EF2475
:10082300B0702A7BFF7A35793F124949EF24B960CA
:100833000D24FE600E2408700FE4FF024DBDE4FF9B
:10084300024DBD7F01024DBD7F3F024DBD7F3F0283
:100853004DBD7BFF7A357943124949EF24BE7003BE
:10086300020D6624FE601A24FB7003020D661460F9
:100873001514601724FE6018240A702A7F01024DA4
:10088300BD7F4F024DBD7F01024DBD7F4F024DBD68
:10089300301407E4FF12000380057F01120003AD4B
:1008A300677F20024CEB7F3F024DBD7BFF7A35799A
:1008B30045124949EF24BC602B1470030209CA2472
:1008C300F97003020A6124F97003020AB214700377
:1008D300020AD424FE7003020AE824136003020B05
:1008E300070212B2756E1974342561F8E6FFB45F1E
:1008F30004E56E70F2EFB45F12E56E700E7642E5BA
:1009030068B40A05E4F568800205687BFF7A3579E7
:100913004D124949EF24B870030209C3240660034A
:100923000209BEE4FF124D81E4FD7FD0124A60123A
:100933004D81E4FD7FD1124A60124D817F01124D3A
:1009430081E4FD7FD2124A60124D81E4FD7FD31210
:100953004A60124D817F02124D81E4FD7FD4124A19
:1009630060124D81E4FD7FD5124A60124D817F03F1
:10097300124D81E4FD7FD6124A60124D81E4FD7F62
:10098300D7124A60124D817F04124D81E4FD7FD856
:10099300124A60124D81E4FD7FD9124A60124D81E3
:1009A3007F05124D81E4FD7FDA124A60124D81E426
:1009B300FD7FDB124A60124D8180057F3F124DBDE2
:1009C300AD677F2E024CEB7BFF7A35794D12494997
:1009D300EF24BE7003020A5A24EC607B240E70726B
:1009E3007F0D124D817F0A124D81E4F56AF56BAFDD
:1009F3006BE4FD124A60E4FD12475E056BE56B7024
:100A030002056AC394FFE56A940040E3E4FD7FFFB7
:100A1300124A60E4FD12475E7F0D124D817F0A1278
:100A23004D81E4F56AF56BAF6B7D02124A60E4FD1C
:100A330012475E056BE56B7002056AC394FFE56AB6
:100A4300940040E37D027FFF124A60E4FD12475E9B
:100A530080057F3F124DBDAD677F2E024CEB7BFFC0
:100A63007A357951124A94E4F58EF508E4F509E5EF
:100A73002775F00CA424002509F8E2FF124D810527
:100A830009E509C3940C40E7E527700575270B803A
:100A93000215277BFF7A357951124A940508E50838
:100AA300C3940C40C7758E02AD677F2E024CEB7565
:100AB3002CF0A82CE2543FF576E4FDAF7612475EA6
:100AC300752CF1A82CE264F8F576E4FDAF760247C5
:100AD3005E123969AF21124D81AF20124D81AD678E
:100AE3007F2E024CEB7BFF7A357954124949BF4381
:100AF3000E752CF9A82CE2F5767D2EFF02475E7F5A
:100B03003F024DBD7F3F024DBD7BFF7A35795612C3
:100B13004949BF5203024C6D7F3F024DBD750941E8
:100B23007BFF7A357958124949EF24BB601924F8C1
:100B3300602024FB600E24FE601024126003020C6C
:100B430081024EA6024F1D750945E509B44103759F
:100B53000954E509B4410375094D7508417BFF7AD2
:100B630035795E124949EF24A9600A24056003021E
:100B73000C7C750852E50864526003750857123EF1
:100B83005BEF64016003020C77852843123E5BEF41
:100B930064016003020C72852844123E5BEF64011A
:100BA3006003020C6D852851E508B45710123E5BB3
:100BB300BF010585285380057F3F024DBDE509240C
:100BC300B37003020C6324F97003020C5E240F60FC
:100BD30003020C68E543540125E0F557E508645228
:100BE3007038F528E528C395515013E5442528FFAF
:100BF300AD57124A60E4FD12475E052880E6E543DF
:100C03005480F52864806003020D66E5442551FF96
:100C1300AD57124A60E4FD02475E756201E4F528B0
:100C2300E528C395515015E5442528FFAB57AD532F
:100C3300124B82EF7002F562052880E4E54354808D
:100C4300F528B48011E5442551FFAB57AD53124B42
:100C530082EF7002F562AF62024DBDE50864522275
:100C6300E5086452227F3F024DBD7F3F024DBD7FA9
:100C73003F024DBD7F3F024DBD7F3F024DBD7F3FD4
:100C8300024DBD7BFF7A357961124949EF24B76084
:100C93003224F2606524156003020D1F123E5BBF10
:100CA3000121E4FDAF28124A608F74E574C39420D8
:100CB3005003124D81AD67AF74124CEB7460257411
:100CC300F574227BFF7A357900124949EF6453703A
:100CD30029F58E7F20124D81789EE6FF124D817F8C
:100CE30020124D81789EE6FFE4FD12475E789EE672
:100CF300FFAD67124CEB758E0222123E5BBF011CE7
:100D03007B007A007977E4F510AF281244B0AF780E
:100D1300AE77122FD8AD677F2E024CEB7F3F024D8B
:100D2300BD7BFF7A357965124949EF6442702A1217
:100D33003E5BEF64017022852851123E5BBF0119AF
:100D4300E4FBAD28AF51124B82BF010575285880D3
:100D530003752845AF28024DBD7F3F024DBD7F3F40
:030D6300124DBD71
:010D6600226A
:104AC600E52704FDE4FF1247F1752CF0A82CE2540B
:104AD60008F576B4080B7BFF7A357967124A94801D
:104AE600097BFF7A35797C124A94AD677F2E024C9A
:014AF600EBD4
:100D670074342561F8E6FF645F70030212B175669B
:100D7700FF8F73765FE561B40A05E4F561800205CC
:100D870061756220E5731206ED0F8F230EE32B0EBC
:100D9700E02D0DC7410E01420E3B430E57470E9102
:100DA7004B0E944D0ECE500ED1520ED4530ED75437
:100DB7000EDA550EDD560FEA5711A3590000129CA3
:100DC700E52704FDE4FF1247F1E55C6401600312C7
:100DD70042B9E55CB4011BE56764366005E567B4B5
:100DE700370A1242B9EF7004FF124DBD7567300222
:100DF7004C8F756738E4FF024DBDE52704FDE4FF1E
:100E07001247F1E55C640160031242B9E55CB40185
:100E17001BE56764366005E567B4370A1242B9EF28
:100E27007004FF124DBD756730024CAE756738E42C
:100E3700FF024DBDE52704FDE4FF1247F1E55CF431
:100E470060067567300249F2756738E4FF024DBDE9
:100E5700E52704FDE4FF1247F1E55C640160031236
:100E670042B9E55CB4011BE56764366005E567B424
:100E7700370A1242B9EF7004FF124DBD7567300291
:100E87003ACB756738E4FF024DBD021B49E52704DD
:100E9700FDE4FF1247F1E55C640160031242B9E526
:100EA7005CB4011BE56764366005E567B4370A1271
:100EB70042B9EF7004FF124DBD756730024A2975BC
:100EC7006738E4FF024DBD022DB40249BA024EC491
:100ED70002461F020713024AC675622DC2A9C2AA9B
:100EE7007F0D124D817F0A124D817BFF7A357991F3
:100EF700124A94123E5B85282DE562642D6007E453
:100F0700FDAF2D12475E123E5B85282EE562642DEC
:100F17006007E4FDAF2E12475E123E5B85282FE582
:100F270062642D6007E4FDAF2F12475E123E5B85BA
:100F37002830E562642D6007E4FDAF3012475E128A
:100F470041D47BFF7A357997124A94E4FDAF6C124E
:100F5700475EE4FDAF4212475EAB46AA47A9481277
:100F6700044EFFE4FD12475EAB46AA47A94890002E
:100F770001120467FFE4FD12475E7BFF7A35799D16
:100F8700124A94D2A9D2AA22C2A9C2AA124CCD8FC0
:100F97002D124CCD8F2E124CCD8F2F124CCD8F3062
:100FA7001241D43017FDC217C299856C993017FDCD
:100FB700C217C2998542993017FDC217C299AB462D
:100FC700AA47A94812044EF5993017FDC217C299CE
:100FD700AB46AA47A948900001120467F599D2A920
:100FE700D2AA227F0D124D817F0A124D817BFF7A93
:100FF7003579A1124A94E4F56AF56BAF6B7D02125D
:101007004A60E4FD12475E056BE56B7002056AC333
:101017009402E56A940040E37F0D124D817F0A1226
:101027004D817BFF7A3579A7124A94756A00756BF3
:1010370002AF6B7D02124A60E4FD12475E056BE565
:101047006B7002056AC39404E56A940040E37F0D60
:10105700124D817F0A124D817BFF7A3579AD124A95
:1010670094756A00756B06AF6B7D02124A60E4FDEA
:1010770012475E056BE56B7002056AC39408E56A63
:10108700940040E37F0D124D817F0A124D817BFF53
:101097007A3579B3124A94756A00756B12AF6B7D16
:1010A70002124A60E4FD12475E056BE56B700205AC
:1010B7006AC39414E56A940040E37F0D124D817F63
:1010C7000A124D817BFF7A3579B9124A94756A0005
:1010D700756B20AF6B7D02124A60E4FD12475E0517
:1010E7006BE56B7002056AC39422E56A940040E3DE
:1010F7007F0D124D817F0A124D817BFF7A3579BFB3
:10110700124A94756A00756B22AF6B7D02124A60B2
:10111700E4FD12475E056BE56B7002056AC3942414
:10112700E56A940040E37F0D124D817F0A124D81DD
:101137007BFF7A3579C5124A94756A00756B26AFBD
:101147006B7D02124A60E4FD12475E056BE56B702A
:1011570002056AC39428E56A940040E37F0D124DA7
:10116700817F0A124D817BFF7A3579CB124A9475BC
:101177006A00756B32AF6B7D02124A60E4FD12475D
:101187005E056BE56B7002056AC39434E56A9400EB
:1011970040E37F0D124D817F0A024D817BFF7A3537
:1011A70079D1124949EF24B870057551208003E4BD
:1011B700F551123E5B852843123E5B8528447BFF31
:1011C7007A3579D4124949EF24B7604124F970037D
:1011D70002126824F8605E24176003021297E55133
:1011E7002406FF7B02AD43124B82E5512407FF7BA8
:1011F70002AD44124B82E551240CFF854412AB43E8
:10120700E4FD124DE8121DC17F01024DBD7B02AD09
:1012170043AF51124B82E55104FF7B02AD44124BA1
:1012270082E5512404FF854412AB43E4FD124DE8E7
:101237007F01024DBDE5512402FF7B02AD43124BF6
:1012470082E5512403FF7B02AD44124B82E5512412
:1012570006FF854412AB43E4FD124DE87F01024DC2
:10126700BDE5512412FF7B02AD43124B82E55124A9
:1012770013FF7B02AD44124B82E5512418FF8544CE
:1012870012AB43E4FD124DE8121DC17F01024DBDB3
:10129700E4FF024DBD7F3F124D81E52704FDE4FFCA
:0B12A7001247F1AD677F3F124CEB22B5
:074ED2007F011200037F0ABB
:074ED9008F6EE56E70FC22F4
:08000300EF24FF92A2921422E7
:063B74007B617D7D7F48AE
:103B7A008F0D8B0E7F01124ED98D6EE50D24B0602C
:103B8A005624FE606824FC601E240E7068E4F51258
:103B9A00FBFD7F23124DE8E56C5404F50D640460C7
:103BAA0054E56E70E8804EE4F512FBFD7F03124D7A
:103BBA00E8E56C5401F50DE5607010752CF1A82C40
:103BCA00E25404F576B40403750D01E50D64016051
:103BDA0024E56E70D2801E7F0112438DEF3395E08B
:103BEA00FEEF64804E700EE56E70EC8008E55F6053
:103BFA0004E56E70F8E56E700EF58E789EA60E7569
:0A3C0A008E02756742FF227F01223F
:1042B9007B6C7D807F52123B7AEF7002FF22123BAA
:1042C90074EF7002FF22E4F55AD2A9D2AA7F011233
:1042D9000003124836EF7005755A288028124E26B9
:1042E900756EFF122C9CBF0119C213124E12EF708A
:1042F90002F56EE56E70F4124E12EF6008755A50B1
:104309008003755A3CE55A6009755C027567387F08
:0B4319000022755C017567307F0122F7
:104C4900E57264087013752CF1A82CE25408F57606
:104C5900B408037F01220242B9E55060037F0122B3
:044C69001242B92218
:1015F600E4F509D2157D027F20123C147B6C7D80B8
:101606007F52123B7AEF7002FF22123B74EF700298
:10161600FF2230130B1242B9EF7005756738FF22AF
:10162600752CF1A82CE25401F576B4010B1242B9DF
:10163600EF7005756738FF22752CF1A82CE254016E
:10164600F576B401067567317F0022752CF1A82C5A
:10165600E25404F576700D7F431237A9EF700575D5
:101666006736FF22752CF1A82CE25408F576700B2C
:101676001242B9EF7005756738FF22E565B450145C
:10168600AF4512438D8F08E508B41008752CF4A8F1
:101696002CE56DF2E565B45208755F19AF6D124D14
:1016A600D3856A3F856B407F4A124450E56524BE68
:1016B600605224F9605424FA604A24FD6021240211
:1016C6007069756EFF7F0112438DEF5480F562B429
:1016D6008004E56E70EFE56E700575674BFF22E4DA
:1016E600F5080508AF6D123A22BF01037508F0E54B
:1016F60008C3940440ECE50864F060037F0022759B
:10170600690180277567317F0022E4F58E7892E5BE
:1017160070F208E571F27890E2FE08E2FFF47002DA
:10172600EEF460048E708F71758E027508300509AF
:10173600E509D39401401DE565B44918E4F58E78B2
:1017460092E2FE08E2FF8E70F5717890EEF208EFF5
:10175600F2758E02E4FF1247A8EF7002FF22752C85
:10176600F1A82CE25401F5767008750832124ED2B3
:1017760080347F03124ED9E56564497026124ED235
:10178600E4FF1200037F05124ED9E4F512FBFD7F3C
:1017960003124DE8E4F58E7890E532F208E533F26F
:1017A600758E02124ED27F431237A9EF7002FF22C6
:1017B600752CF1A82CE25401F5767009E50864321F
:1017C6006003750839E508B43209E56564496003C4
:1017D600750905E509C394025012E50864397003DA
:1017E600021731E50864327003021731E56524AE4D
:1017F60060092402700A124E4E8005AF6D124EB675
:10180600E508643060347F011200033000107B006D
:101816007A00793FE4F5107F061244B0800E7B0013
:101826007A00793FE4F5107F6E1244B07572087F36
:101836004A1244508508677F0022E565B449087559
:1018460050FFE4F5728003757208E5656452704ACC
:10185600E56D24FE701B7B007A00793FE4F5107F6E
:10186600761244B07550FFE4F5727F4A12445080F8
:10187600293000107B007A00793FE4F5107F0612CC
:1018860044B0800E7B007A00793FE4F5107F6E123B
:1018960044B07572087F4A124450E56764306003AD
:0518A6007F00227F011C
:0118AB00221A
:10243000C2157D027F20123C1430130B1242B9EFFB
:102440007005756738FF22752CF1A82CE25401F550
:10245000767005756746FF227F431237A9EF700239
:10246000FF22123B74EF7002FF22752CF1A82CE2C0
:102470005408F5767011124C49EF700B1242B9EF07
:102480007005756738FF22E565B45014AF451243F7
:102490008D8F08E508B42008752CF4A82CE56DF2A2
:1024A000E565B45208755F19AF6D124DD3856A3F6B
:1024B000856B407F4A124450E56524BE605824F97C
:1024C000700302254C24FA607924FD602424026004
:1024D00003022551756EFF7F0112438DEF5480F585
:1024E00062B48004E56E70EFE56E700575674BFFB2
:1024F00022E4F5080508AF6D123A22BF0103750802
:10250000F0E508C3940440ECE50864F060037F0044
:1025100022750830803B30001F756EFF7F0112432B
:102520008DEF5480F562B48004E56E70EFE562B41F
:10253000800675674B7F0022E569B40114124AF7E3
:10254000800FE569B4010A12222E8005E4F570F5CA
:10255000717F011247A8EF7002FF22E4FF1200030F
:102560007F08124ED9750830E565644F6005E56552
:10257000B44210752CF1A82CE25401F576B4010395
:102580007508497F431237A9EF7002FF227F0112BD
:102590000003752CF1A82CE25401F576B401057501
:1025A000674D1F22E56524AE60092402700A124EB1
:1025B0004E8005AF6D124EB63000107B007A007968
:1025C0003FE4F5107F061244B0800E7B007A00795C
:1025D0003FE4F5107F6E1244B07572087F4A1244D2
:0E25E00050E508B449067567497F00227F0167
:0125EE0022CA
:104BD6007F011230E5EF7002FF221215F6EF700228
:104BE600FF227F021230E5EF7002FF22122430EF1F
:074BF6007002FF227F012283
:054E9600124E9BD291B9
:0B4E9B000000000000000000000022EA
:104E7400D291124E9BD290124E9BC290124E9BC264
:024E8400912279
:084F2600C290124E96D29022B7
:0D4EE000D290124E96A2909231C291A23152
:014EED0022A2
:0A4F1300A2319290124E96C2912234
:104BAD00124EE0921F124EE0921E124EE0921D1216
:104BBD004EE0921C124EE0921B124EE0921A124ED3
:094BCD00E09219124EE092182248
:08487A00124E74EB24A0F5239B
:10488200A21F9231124F13A21E9231124F13A21D78
:104892009231124F13A21C9231124F13A21B92316A
:1048A200124F13A21A9231124F13A2199231124FC0
:0B48B20013A2189231124F13024EE0C7
:104D8F00E55870FC12487A8F231248828D231248FF
:084D9F0082124F267558032211
:104A6000AE8EE4F58EE55870FC124E74ED12487E61
:104A70008F23124882124E74ED24A1F5231248822E
:104A8000124BADD230A2309231124F13124F268EFC
:034A90008EAF23C3
:014A93002200
:04470F00AC05A90745
:10471300858E0AE4F58EFAEAC39C5011E92AFFADAF
:1047230003124A6074922AF8A6070A80EABC022799
:104733007892E6FF789F860308E6FA08E6F9EF1217
:1047430004947893E6FF789F860308E6FA08E6F96F
:0A475300900001EF1204A6850A8E03
:01475D002239
:0844B0008F0C8B0D8A0E890FA1
:1044B800858E11E4F58EFCE50C2CFFAD10124A60D8
:1044C80074922CF8A6070CBC02ED7892E6FF789F50
:1044D800860308E6FA08E6F9EF1204947893E6FFF3
:1044E800789F860308E6FA08E6F9900001EF1204BF
:1044F800A678A2E6FF08E6AB0DAA0EA90FCF8FF0AB
:0645080012052F85118E43
:01450E00228A
:064B8200AE07AC03AA051A
:104B8800A98EE4F58EAF06AD02AB04124D8FAD04CD
:104B9800124A60E523B50205898E7F0122898E7548
:044BA80067337F00F0
:014BAC0022E6
:06456B008F0B8D0C8B0D7F
:10457100858E0FE4F58EE50CB40219789F86030849
:10458100E6FA08E6F912044E7892F6900001120458
:10459100677893F6E4F50EE50EC3950C5020E50B14
:1045A100250EFF7492250EF8E6FDAB0D124B82EF3E
:1045B1007008850F8E756733FF22050E80D9850F30
:0345C1008E7F01E9
:0145C40022D4
:103DD300AE8EE4F58EEDD3940840027D08E558706D
:103DE300FC12487A8F23124882E4FCECC39D500DE9
:103DF30074922CF8E6F5231248820C80EE124F26BB
:103E0300755803E55870FC12487A8F2312488212C2
:103E13004E74EB24A1F523124882E4FCECC39D50BD
:103E230027124BAD74922CF8E523666003ED04FC76
:103E3300ED14FFECC39F4004D2308002C230A230A5
:103E43009231124F130C80D4124F268E8EECD39DD9
:073E530040037F00227F0104
:013E5A002245
:1048BD00E4FFAE8EF58EFDE55870FC124E74752337
:1048CD00A0124882EDC454F0F523124882E4FCEFA7
:1048DD00C394C04006EFD394D0400675232E1248E2
:1048ED00820F0CBC10E9124F267558030DBD10C771
:0248FD008E8E9D
:0148FF002296
:104E61003234363841530020616C743A00206E654B
:034E7100753A008F
:104D4000E4F58E78A2A60408A605758E027D0212EF
:0B4D5000456BBF01037F01227F0022A2
:03000E007F01224D
:1045C500AE03E4F58E78A2A60E08A60F789F8603A3
:1045D50008E6FA08E6F912044E7892F69000011200
:1045E50004677893F608A60508A60608A60C08A68B
:1045F5000D78A2A61008A61112044E7898F6900020
:10460500011204677899F6758E02E4FB7D08123D68
:0A461500D3BF01037F01227F0022C2
:102ECA00E55924FE6003022FD2750C30750D30755A
:102EDA000E3F750FD075105F75115C7B017D527FB7
:102EEA00201245C5EF7002FF22750C30750D307542
:102EFA000E34750F887510687511D87B017D497F6E
:102F0A00801245C5EF7002FF22750C30750D3075C1
:102F1A000E15750F887510767511D07B807D50E47B
:102F2A00FF1245C5EF7002FF22750C30750D30E4B3
:102F3A00F50EF50F7510847511987B017D4F7F7022
:102F4A001245C5EF7002FF22750C30750D30750EF3
:102F5A003F750FD075108D75114C7B027D527F28FD
:102F6A001245C5EF7002FF22750C30750D30750ED3
:102F7A000B750FB87510767511D07B037D527F30B3
:102F8A001245C5EF7002FF22750C30750D30750EB3
:102F9A0015750F7C7510767511D07B047D527F38BC
:102FAA001245C5EF7002FF22750C30750D30750E93
:102FBA001C750FC07510767511D07B017D427F6834
:0E2FCA001245C5EF7005FF227F00227F012215
:104C2300E4FBFD7FF4124B82BF0115E4F552FBFD5B
:104C33007FF5124B82BF0105E4F54980067F002210
:064C43007F00227F012228
:1033F0007B027D117F60124B827B027D077F611211
:103400004B827B027D217F62124B827B02E4FDFFB7
:10341000124B827B027D647F01124B827B027D0214
:103420007F02124B827B027DFF7F03124B827B0265
:103430007D037F06124B827B027DFF7F07124B824A
:103440007B027DF27F0B124B827B027D087F0C1288
:103450004B827B02E4FD7F0D124B827B02E4FD7FF9
:103460000E124B827B027D397F12124B827B027DD2
:10347000037F13124B827B02E4FD7F20124B827B81
:10348000027D017F21124B827B027D017F22124B44
:10349000827B027DFF7F23124B827B027D017F2690
:1034A000124B827B027DFF7F27124B827B027DF2D3
:1034B0007F2B124B827B027D097F2C124B827B0279
:1034C000E4FD7F2D124B827B02E4FD7F2E124B82A6
:1034D0007B027D497F32124B827B027D047F331257
:0534E0004B827F012278
:102A5200E4FBFD7FD0124B82E4FB7D4B7FD1124B16
:102A620082E4FB7D017FD2124B82E4FB7D047FD3A3
:102A7200124B82E5216076E4FB7D017FD4124B820A
:102A820030095F300A51300B43300C35300D27309E
:102A92000E19300F0BE4FB7D087FD5124B82805D4F
:102AA200E4FB7D077FD5124B828052E4FB7D067FDB
:102AB200D5124B828047E4FB7D057FD5124B828085
:102AC2003CE4FB7D047FD5124B828031E4FB7D0325
:102AD2007FD5124B828026E4FB7D027FD5124B828A
:102AE200801BE4FB7D017FD5124B828010E4FBFD4D
:102AF2007FD4124B82E4FBFD7FD5124B82E4FB7D37
:102B0200017FD6124B82E4FB7D047FD7124B82E514
:102B12002054C3603EE4FB7D017FD8124B8230011A
:102B22002730061930070BE4FB7D047FD9124B8254
:102B32008031E4FB7D037FD9124B828026E4FB7D4A
:102B4200027FD9124B82801BE4FB7D017FD9124B9D
:102B5200828010E4FBFD7FD8124B82E4FBFD7FD91B
:102B6200124B82E4FB7D047FDA124B82E4FB7D048C
:052B72007FDB124B8225
:012B7700223B
:10467000122ECAEF7002FF2212000EEF7002FF220C
:10468000E4FB7D047FEC124B82E4FB7D0A7FBC12CD
:104690004B82E4FB7D687C427F9E124D40122A5281
:1046A000EF7002FF22124C23EF7002FF221233F050
:1046B000EF7002FF22122789EF7002FF227F012292
:1025EF00750A01D216E4FF1247A8EF7002FF227599
:1025FF005DFF7550FF75092D74342561F8E6645F32
:10260F00703BE55D64016004E5667010E4F55DFD07
:10261F00FF123C147560037F01120003E550640143
:10262F006007E566600302274BE4F550FD7F20123B
:10263F003C147556037F0112000302274B7BFF7A70
:10264F004E79611249498F09E50924CC700302269E
:10265F00DD24FE700302271224FE603C2406600373
:10266F0002274B74102571F571E43570F570D3E5C1
:10267F00719468E570944240067570427571688573
:10268F00703F8571407F611237A9EF7005F50A75AC
:10269F000945755DFF02274BC3E5719410E57094F2
:1026AF00005007E4F570F571800C74F02571F57129
:1026BF0074FF3570F57085703F8571407F611237FB
:1026CF00A9EF7005F50A750945755DFF806E74FCFD
:1026DF00256BF56B74FF356AF56AC3E56B94C0E53E
:1026EF006A945D5006756A5D756BC0856A3F856B30
:1026FF00407F61124450EF7005F50A75094575501A
:10270F00FF80397404256BF56BE4356AF56AFEAF0B
:10271F006BE4FCFD7B307A8EF9F8C3120679500614
:10272F00756A8E756B30856A3F856B407F61124489
:10273F0050EF7005F50A7509457550FFE5096453AB
:10274F006009E50964416003022607C216E50A64C1
:10275F00017021E509B45319E4FBAD71AC70AF41C1
:10276F00124D40E5412406FFE4FBAD6BAC6A124D00
:09277F00400242B91242B97F0088
:01278800222E
:10415A008F09E4FD7FF4124A608F527BFF7A4E7911
:10416A0068124A94C374FF9552FFE49400FE122F1A
:10417A00D8E552D3949B400CE4FB7D9B7FF4124B11
:10418A008275529BE5527008E509B4FF03E4F5090C
:10419A00E552B49B08E509B40103E4F509E50925EC
:1041AA0052F552E4FBAD527FF4124B82EF7002FFDC
:1041BA00227BFF7A4E796E124A94C374FF9552FF9E
:0A41CA00E49400FE122FD87F0122BA
:103F64008F09E4FD7FF5124A608F497BFF7A4E7911
:103F740068124A94E549D3949B40057F30124D81E1
:103F8400C374FF9549FFE49400FE122FD8E54970ED
:103F940008E509B4FF03E4F509E549B4FF08E509B8
:103FA400B40103E4F509E5092549F549E4FBAD4904
:103FB4007FF5124B82EF7002FF227BFF7A4E796EFF
:103FC400124A94E549D3949B40057F30124D81C336
:0F3FD40074FF9549FFE49400FE122FD87F01225D
:0C4F0700474F4F443A00204241443A001A
:10222E00E4F569FD7FC0124A608F76E50BF4601409
:10223E00050BE4FBAD0B7FC0124B82BF01037F0188
:10224E00227F0022E4FD7FC1124A608F0BE50BF462
:10225E006014050BE4FBAD0B7FC1124B82BF010373
:10226E007F01227F0022E4FD7FC2124A608F0BE5C0
:10227E000BF46014050BE4FBAD0B7FC2124B82BF57
:10228E0001037F01227F0022E4FD7FC3124A608F8B
:10229E000BE50BF46014050BE4FBAD0B7FC3124B87
:1022AE0082BF01037F01227F0022E4FD7FC4124A18
:1022BE00608F0BE50BF46014050BE4FBAD0B7FC4D4
:1022CE00124B82BF01037F01227F0022E4FD7FC5F6
:1022DE00124A608F0BE50BF46014050BE4FBAD0B9B
:1022EE007FC5124B82BF01037F01227F0022E4FDD6
:1022FE007FC6124A608F0BE50BF46014050BE4FBEE
:10230E00AD0B7FC6124B82BF01037F01227F0022DD
:10231E00E4FD7FC7124A608F0BE50BF46014050BCA
:10232E00E4FBAD0B7FC7124B82BF01037F01227FFF
:10233E000022E4FD7FC8124A608F0BE50BF4601497
:10234E00050BE4FBAD0B7FC8124B82BF01037F016F
:10235E00227F0022E4FD7FC9124A608F0BE50BF449
:10236E006014050BE4FBAD0B7FC9124B82BF01035A
:10237E007F01227F0022E4FD7FCA124A608F0BE5A7
:10238E000BF46014050BE4FBAD0B7FCA124B82BF3E
:10239E0001037F01227F0022E4FD7FCB124A608F72
:1023AE000BE50BF46014050BE4FBAD0B7FCB124B6E
:1023BE0082BF01037F01227F0022E4FD7FCC124AFF
:1023CE00608F0BE50BF46014050BE4FBAD0B7FCCBB
:1023DE00124B82BF01037F01227F0022E4FD7FCDDD
:1023EE00124A608F0BE50BF46035050BE4FBAD0B69
:1023FE007FCD124B82BF0124750900750AC0AF0A4A
:10240E00E4FBFD124B82050AE50A70020509C3942E
:10241E00CDE5096480948040E57F01227F00227F14
:01242E0001AC
:01242F00228A
:104AF700E4F569FD7FCE124A60EF3395E0FEEFF4EF
:104B07007002EEF460170FBF00010EAD07E4FB7FE4
:0F4B1700CE124B82BF01037F01227F00227F015C
:014B2600226C
:1012B200E4F58E789A1206D400000000E4FD7FCD9A
:1012C200124A60EF3395E0FEFDFC789A1206C87868
:1012D2009A12068FE47BF37A0CF9F812054E789A8B
:1012E2001206C8789A1206ABC000C001C002C00341
:1012F200E4FD7FC0124A60EF3395E0FEFDFCD003AF
:10130200D002D001D000EB2FFFEA3EFEE93DFDE81E
:101312003CFC789A1206C8789A1206ABC000C0014B
:10132200C002C003E4FD7FC1124A60EF3395E0FEC4
:10133200FDFCD003D002D001D000EB2FFFEA3EFE2D
:10134200E93DFDE83CFC789A1206C8789A1206AB91
:10135200C000C001C002C003E4FD7FC2124A60EFB8
:101362003395E0FEFDFCD003D002D001D000EB2F7C
:10137200FFEA3EFEE93DFDE83CFC789A1206C87899
:101382009A1206ABC000C001C002C003E4FD7FC3D5
:10139200124A60EF3395E0FEFDFCD003D002D0018B
:1013A200D000EB2FFFEA3EFEE93DFDE83CFC789AD7
:1013B2001206C8789A1206ABC000C001C002C00370
:1013C200E4FD7FC4124A60EF3395E0FEFDFCD003DA
:1013D200D002D001D000EB2FFFEA3EFEE93DFDE84E
:1013E2003CFC789A1206C8789A1206ABC000C0017B
:1013F200C002C003E4FD7FC5124A60EF3395E0FEF0
:10140200FDFCD003D002D001D000EB2FFFEA3EFE5C
:10141200E93DFDE83CFC789A1206C8789A1206ABC0
:10142200C000C001C002C003E4FD7FC6124A60EFE3
:101432003395E0FEFDFCD003D002D001D000EB2FAB
:10144200FFEA3EFEE93DFDE83CFC789A1206C878C8
:101452009A1206ABC000C001C002C003E4FD7FC700
:10146200124A60EF3395E0FEFDFCD003D002D001BA
:10147200D000EB2FFFEA3EFEE93DFDE83CFC789A06
:101482001206C8789A1206ABC000C001C002C0039F
:10149200E4FD7FC8124A60EF3395E0FEFDFCD00305
:1014A200D002D001D000EB2FFFEA3EFEE93DFDE87D
:1014B2003CFC789A1206C8789A1206ABC000C001AA
:1014C200C002C003E4FD7FC9124A60EF3395E0FE1B
:1014D200FDFCD003D002D001D000EB2FFFEA3EFE8C
:1014E200E93DFDE83CFC789A1206C8789A1206ABF0
:1014F200C000C001C002C003E4FD7FCA124A60EF0F
:101502003395E0FEFDFCD003D002D001D000EB2FDA
:10151200FFEA3EFEE93DFDE83CFC789A1206C878F7
:101522009A1206ABC000C001C002C003E4FD7FCB2B
:10153200124A60EF3395E0FEFDFCD003D002D001E9
:10154200D000EB2FFFEA3EFEE93DFDE83CFC789A35
:101552001206C8789A1206ABC000C001C002C003CE
:10156200E4FD7FCC124A60EF3395E0FEFDFCD00330
:10157200D002D001D000EB2FFFEA3EFEE93DFDE8AC
:101582003CFC789A1206C8789A1206ABC000C001D9
:10159200C002C003E4FD7FCD124A60EF3395E0FE46
:1015A200FDFCD003D002D001D000EB2FFFEA3EFEBB
:1015B200E93DFDE83CFC789A1206C87F0D124D8188
:1015C2007F0A124D817BFF7A4F7907124A941220CB
:1015D2001F7BFF7A4F790D124A94E4FD7FCE124AA7
:1015E20060EF3395E0FEFDFC789A1206C812201FC8
:0415F200758E0222CE
:104C6D00750A00750BC0AF0BE4FBFD124B82050BF3
:104C7D00E50B7002050AC394D0E50A648094804068
:014C8D00E541
:014C8E002203
:1041D400C2A1E4FFFE742D2FF8E6F513E4FDFCC242
:1041E40096E51330E704D2948002C294E51325E0E7
:1041F400F513D29630B4034313010DBD00010CED49
:1042040064084C70DAEE7033EF14600F146011140C
:10421400601B2403702585136C8020851342801B4A
:10422400AB46AA47A948E513120494800EAB46AAEC
:1042340047A948900001E5131204A60FBF00010E20
:08424400EF64044E708FD2A15B
:01424C00224F
:104DE800C2A9C2AA8F2D8D2E8B2F8512301241D4C5
:054DF800D2A9D2AA229D
:10424D008F17AF03C2A985172D8D2E8F2F851A308D
:10425D00C2A1E4FF742D2FF8E6F517E4F51AC29606
:10426D00E51730E704D2948002C294E51725E0F5F6
:10427D0017D29630B403431701051AE51AB408DEB8
:10428D00EF24FD601004701BAB29AA2AA92BE5179A
:10429D00120494800EAB29AA2AA92B900001E517D0
:0C42AD001204A60FBF04ADD2A1D2A922BA
:101DC100E4F58E7879F67879E6FFD3942040030222
:101DD100201BEF2412FF7D02124A60EF540F787A24
:101DE100F618E62412FF7D02124A60EF54F0787B68
:101DF100F6E6FFC4540FF67879E62406FF7B027DF0
:101E01000212470F78A2E6FE08E6FF787CA60608D4
:101E1100A607787BE6FF18E6C39FFDE49400FCE487
:101E21001203368F0F8E0E8D0D8C0C7F007E007D80
:101E3100007C401236C8E4FBFAF9784312011EC057
:101E410004C005C006C007787CE6FC08E6FDEC127C
:101E51000336D003D002D001D000120227788612B7
:101E610006C8788A1206D4BF800000E47880F6089C
:101E7100F67884F6087680787EF608F6787EE6FEB7
:101E810008E6FFD3940DEE648094804003021FE0C6
:101E9100EF2403FDE43EFC1203368F0F8E0E8D0DF1
:101EA1008C0C7F007E007D007C401236C878861243
:101EB10006AB12011E12036F7882EEF608EFF6D31D
:101EC100947FEE648094805003021FD518E66480ED
:101ED10094814003021FD5787FE62403FD18E43680
:101EE100FC1203368F0F8E0E8D0D8C0C7F007E0041
:101EF1007D007C401236C8C004C005C006C007780A
:101F010082E6FC08E6FDEC120336D003D002D001D4
:101F1100D000120227788E1206C8788A1206ABC04A
:101F210000788612068FD000120029124EEEC004EE
:101F3100C005C006C007788A1206ABC000788E12B1
:101F4100068FD000120029124EEEA804A905AA0698
:101F5100AB07D007D006D005D0041202C4400FE46D
:101F6100FFFEFDFC788A1206AB1202C45066787F30
:101F7100E62403FD18E436FC1203368F0F8E0E8D16
:101F81000D8C0C7F007E007D007C401236C8788667
:101F91001206AB12011EE4FBFA79BE784212011E51
:101FA100E4FBFA79C8784212022712036F7882EEB5
:101FB100F6FA08EFF6FB788E12068F788A1206C8B9
:101FC100787EE6FE08E6FF08A60608A6077884A63E
:101FD1000208A603787F06E618700106021E7D78C6
:101FE10079E6240BFF7885E6FD7B02124B82787936
:101FF100E6240CFF7881E6FD7B02124B827879E6BC
:102001002412FF7885E6FB7881E6F512E4FD124D96
:0D201100E87879742026F6021DC7758E024E
:01201E00229F
:1032F1007D027F60124A608F2E7D027F61124A60DB
:103301008F2F7D027F62124A608F30853012AB2F82
:10331100AD2E7F7E124DE8E4F5087B027D02AF08F9
:1033210012470FE5082404FF789F860308E6FA0890
:10333100E6F912044EFBC003789F860308E6FA08FB
:10334100E6F9900001120467F512D003E4FD124D75
:10335100E8E5082406FFE4F512FBFD124DE8E50857
:103361002406FF7B027D0212470FE508240CFF783B
:103371009F860308E6FA08E6F912044EFBC00378BB
:103381009F860308E6FA08E6F9900001120467F542
:1033910012D003E4FD124DE8E5082414FFE4F51210
:1033A1007B03FD124DE8E5082412FF7B027D02122A
:1033B100470FE5082418FF789F860308E6FA08E618
:1033C100F912044EFBC003789F860308E6FA08E66B
:1033D100F9900001120467F512D003E4FD124DE8E3
:0E33E10074202508F508D39420500302331BF6
:0133EF0022BB
:104B5600E4F52E75088085082DE50804FF7D021210
:104B66004A608F2F7D02AF08124A608F301241D4FF
:0B4B760005080508E508C394FE40DBBD
:014B81002211
:10278900E4F58E789276110876110876100876109D
:1027990008760608761008761008762E7B027D08E2
:1027A9007F80123DD3EF7005758E02FF227B027D7B
:1027B900087F88123DD3EF7005758E02FF22E478F9
:1027C90092F60876020876030876040876060876F3
:1027D9000708760908760A7B027D087FC0123DD377
:1027E900EF7005758E02FF227892760C08760E0836
:1027F900760F087611087612087614087615087689
:10280900177B027D087FC8123DD3EF7005758E02D4
:10281900FF227892761808761908761B08761C0824
:10282900761E08761F0876200876227B027D087FAF
:10283900D0123DD3EF7005758E02FF227892762370
:10284900087624087626087627087628087629083F
:10285900762A08762C7B027D087FD8123DD3EF704B
:1028690005758E02FF227892762D08762E08762F2E
:102879000876300876310876320876330876347B64
:10288900027D087FE0123DD3EF7005758E02FF22AD
:1028990078927635087636087636087637087638A7
:1028A90008763908763908763A7B027D087FE8127E
:1028B9003DD3EF7005758E02FF227892763B08763C
:1028C9003B08763C08763C08763D08763D08763E1E
:1028D90008763E7B027D087FF0123DD3EF700575C7
:1028E9008E02FF227892763E08763F08763F087678
:1028F9003F08763F08763F08763F08763F7B027DA2
:10290900087FF8123DD3EF7005758E02FF22758E90
:04291900027F012216
:104EA600752CF0A82C7402F2752CF7A82C14F2229B
:094F1D00752CF7A82C7402F22295
:104D08003031323334353637383900303132333494
:0C4D1800353637383941424344454600E7
:0C4D7500FAF9F81205D9EF2430F50AFF16
:0E4D8100E55B70FC3017FDC217C2998F9922B6
:10475E00AE05AD07ED54F0F576C4540FF562D39463
:10476E0009500874302562F562800674372562F5AB
:10477E0062AF62124D81EE6004FF124D81ED540F57
:10478E00F562D39409500874302562F56280067480
:0A479E00372562F562AF62024D811B
:064A94008B0A8A0B890C5D
:104A9A00124DFDAC07E4FDC3EC6480F8ED64809828
:104AAA005019AB0AAA0BA90CEDFF3395E08F82F5DA
:0B4ABA0083120467FF124D810D80DCA9
:014AC50022CE
:042FD8008E0A8F0BC3
:102FDC00E4FB7C277D101204DAC3E50B9DFFE50AA8
:102FEC009CFE7C277D101204DAEF2430FA643060EA
:102FFC00060BAF02124D81EA24D0FFE434FFFE7CB5
:10300C00277D101204C8C3E50B9FF50BE50A9EF54E
:10301C000AFEAF0B7C037DE81204DAC3E50B9DFFBF
:10302C00E50A9CFE7C037DE81204DAEF2430FA6496
:10303C003060097B01AF02124D818008BB0105AFE6
:10304C0002124D81EA24D0FFE434FFFE7C037DE8BC
:10305C001204C8C3E50B9FF50BE50A9EF50AFEAFFB
:10306C000B7C007D641204DAC3E50B9DFFE50A9C22
:10307C00FE7C007D641204DAEF2430FA64306009BF
:10308C007B01AF02124D818008BB0105AF02124DCE
:10309C0081EA24D075F064A4FFAEF0C3E50B9FF574
:1030AC000BE50A9EF50AFEAF0B7C007D0A1204DAD2
:1030BC00C3E50B9DFFE50A9CFE7C007D0A1204DA39
:1030CC00EF2430FAFF124D81EA75F00AA4FEC3E535
:0930DC000B9E2410FAFF024D8145
:10201F00E4F58E7BA07A867901F8C000789A1206D3
:10202F008FD0001205D9C000789A12068FD000C346
:10203F00EF9BFFEE9AFEED99FDEC98FC7BA07A8664
:10204F0079017800124D78789A12068FC004C00576
:10205F00C006C007E50A24D0FFE434FFFEE4FCFD10
:10206F007BA07A867901F812054EA804A905AA0665
:10207F00AB07D007D006D005D004C3EF9BFFEE9A75
:10208F00FEED99FDEC98FC789A1206C8E47B107A65
:10209F0027F9F8C000789A12068FD0001205D9C020
:1020AF0000789A12068FD000C3EF9BFFEE9AFEEDD9
:1020BF0099FDEC98FCE47B107A27124D76789A12F2
:1020CF00068FC004C005C006C007E50A24D0FFE490
:1020DF0034FFFE7C277D101204C8E4FCFDAA06AB7A
:1020EF0007D007D006D005D004C3EF9BFFEE9AFEB2
:1020FF00ED9400FDEC9400FC789A1206C8E47BE89E
:10210F007A03F9F8C000789A12068FD0001205D919
:10211F00C000789A12068FD000C3EF9BFFEE9AFE95
:10212F00ED99FDEC98FCE47BE87A03124D76789AF2
:10213F0012068FC004C005C006C007E50A24D0FFF1
:10214F00E434FFFE7C037DE81204C8E4FCFDAA061C
:10215F00AB07D007D006D005D004C3EF9BFFEE9A94
:10216F00FEED9400FDEC9400FC789A1206C8E47B17
:10217F0064FAF9F8C000789A12068FD0001205D9C8
:10218F00C000789A12068FD000C3EF9BFFEE9AFE25
:10219F00ED99FDEC98FCE47B64124D75789A12066C
:1021AF008FC004C005C006C007E50A24D075F064CF
:1021BF00A4FFAEF0E4FCFDAA06AB07D007D006D013
:1021CF0005D004C3EF9BFFEE9AFEED9400FDEC9457
:1021DF0000FC789A1206C8E47B0AFAF9F8C0007876
:1021EF009A12068FD0001205D9C000789A12068F66
:1021FF00D000C3EF9BFFEE9AFEED99FDEC98FCE447
:10220F007B0A124D75789DE6FFE50A75F00AA4FE6C
:0E221F00C3EF9E2410F50AFF124D81758E024A
:01222D00228E
:1047F1008F75BD0C02E4FDE5276D6017E4F58EFFB2
:10480100ED75F00CA424002FF8745FF20FBF0CF0CB
:10481100758E028D27E4F58EE52775F00CA4240032
:104821002575F8E573F2758E02E575B40B04E4F5B0
:044831007522057572
:014835002260
:08494100F5287BFF7A4D79088F
:1049490074342561F8E6FF645F60F58F73765FE57F
:1049590061B40A05E4F56180020561AF750575ADBD
:10496900271247F1AD73124D24EF2401FFE43E4FA6
:084979006003AF73227F0022EE
:104CEB00E4F58EE52775F00CA4240AF8EFF2E5271E
:0D4CFB0075F00CA4240BF8EDF2758E02226A
:023FE3008F0944
:103FE5001249438F0AE50A7005756731FF22E50A14
:103FF50024D01249418F0AE50A7005756731FF2201
:10400500AF287804EF08800123D8FDFFE50A24D006
:104015002F1249418F0AE50A7005756731FF22E5C0
:104025000A24D0F5741249438F0AE50A70057567AD
:1040350031FF22AF747804EF08800123D8FDFFE536
:104045000A24D02FF574E509B40108852851857433
:0B4055004380068528538574447F01DA
:01406000223D
:103E5B007BFF7A4D79131249498F0AE50A70057574
:103E6B006731FF22C3E50A648094BC500EE50A2437
:103E7B00D0F52875F00AA4F5748009E50A24C9F574
:103E8B00287574FF7BFF7A4D79131249498F0AE528
:103E9B000A7005756731FF22C3E50A648094BC5034
:103EAB0020AF287804EF08800123D8FDFFE50A2412
:103EBB00D0FE2FF528E574F4601AE5742EF57480A6
:103ECB0013AF287804EF08800123D8FDFFE50A24FF
:063EDB00C92FF5287F014C
:013EE10022BE
:104CCD0074342561F8E6FF645F60F58F73765FE5F8
:0E4CDD0061B40A05E4F56180020561AF73223F
:104DBD00AE07BE01027E58EE70027E45AF06124D63
:064DCD0081AD67024CEB12
:100026000203DBE86480F8E933E83360110460F02A
:10003600ED33EC337009E8FCE9FDEAFEEBFF220440
:1000460060DED3EB9FEA9EE99DE8C2E78CF0C2F73B
:1000560095F0400CE8CCF8E9CDF9EACEFAEBCFFB07
:100066001203A685D0F05804700320D5B3E80470B7
:10007600075002B2D50203E592D5EC0460F7E4CC52
:10008600C0E0C398F8603B94186008400DD0E0FBD0
:100096000203BDE4FBFAC9FC8028E830E406E4C9A3
:1000A600FBE4CAFCE830E305E4C9CACBFCE8540724
:1000B6006010F8C3E913F9EA13FAEB13FBEC13FC2F
:1000C600D8F130F52FC3E49CFCEF9BFFEE9AFEEDD2
:1000D60099FDD0E0FBEF4E4D4C701222DB0302037C
:1000E600E2EC2CFCEF33FFEE33FEED33FDED30E7B3
:1000F600EB0203BDEF2BFFEE3AFEED39FDD0E0FB40
:1001060050130BBB00030203E5ED13FDEE13FEEFE8
:0801160013FFEC13FC0203BD12
:10011E00EC4D6011E8497017ED33EC3304600DE4DB
:10012E00FCFFFEFD22E933E8330470F80203DB1214
:10013E0003A658046009E4CC248150062850090215
:10014E0003E52840030203E2C0E0EB4A7044B980A5
:10015E0006D0E0FB0203D1EF4E701CBD8008EBFF12
:10016E00EAFEE9FD80EBE98DF0A4FEE5F002020760
:10017E00E9CDF9EAFEEBFFEF89F0A4FCE5F0CE89BC
:10018E00F0A42EFFE435F0CD89F0A42DFEE435F079
:10019E008067EF4E7005BD80D780C3EF8BF0A4ACA7
:1001AE00F0EE8BF0A42CFCE435F0F8EF8AF0A42CE2
:1001BE00E5F038FCE433CB8DF0A42CFCE5F03BF8F5
:1001CE00EE8AF0A42CFCE5F038F8E433CF89F0A4E5
:1001DE002CFCE5F038CF3400CE89F0A42FFFE5F0EB
:1001EE003EFEE433C98DF0A42EFEE5F039CD8AF043
:1001FE00A42FFFE5F03EFEE43DFD33D0E0FB5007BB
:10020E000BBB000F0203E5EC2CFCEF33FFEE33FECD
:06021E00ED33FD0203BDFB
:100224000203E5EC5D046005E8590470030203DB96
:100234001203A6580460F6EC4860F2EC7004FDFE6C
:10024400FF22C860DB2481C85009C39860025006AD
:100254000203E29850CAF582E9294B4A7005AB8241
:100264000203D175F0007C1A7880C3EF9BEE9AEDFF
:1002740099400DC3EF9BFFEE9AFEED99FDE842F025
:10028400DC23ACF0D0E0FFD0E0FED0E0FDAB822078
:10029400E7101BEB60BAEC2CFCEF33FFEE33FEED02
:1002A40033FD0203BDE803F830E705C0F075F00044
:1002B400EF2FFFEE33FEED33FD40B830E7C280AAE6
:1002C40074F8CC6480CCC86480C8F582046043C3ED
:1002D400EB9FF5F0EA9E42F0E99D42F0E89C45F080
:1002E40060305018E5825FFFE582F42B5582FB50A5
:1002F400210ABA001D09B90019088016E5825BFBC2
:10030400E582F42F5582FF50090EBE00050DBD0095
:10031400010CC3EB9FF5F0EA9E42F0E99D42F0E840
:0D0324009C45F06007CC4820E701B3EC22B7
:1003310075F020800E75F010800575F0087D007E47
:10034100007F003392D530D50312066BEC33401099
:10035100EF33FFEE33FEED33FDEC33FCD5F0ED2250
:0E036100E5F0247EA2D513CC92E7CDCEFF228C
:10036F00EDD2E7CD33EC3392D524814006E4FFFE86
:10037F00FDFC22FCE4CFCECDCC24E0501174FF80E5
:10038F00EDC3CC13CCCD13CDCE13CECF13CF047082
:07039F00F030D5DE02066B11
:0D4EEE00ED33EC3360065004EC6480FC22D0
:1036C8008F0B8E0A8D098C08E4FFFEFDFCAB0BAA5C
:1036D8000AA909A8081202C4702CFFFEFDFCAB0F52
:1036E800AA0EA90DA80C1202C460084006E4FFFE49
:1036F800FDFC2274FFF50FF50EF50DF50CAF0FAEBE
:103708000EAD0DAC0C22E4F510F511FFFEFDFCAB7F
:103718000BAA0AA909A8081202C4504BAF0FAE0E93
:10372800AD0DAC0C12036F8E108F11AC10AD11E4FF
:10373800120336C8ECC8C9EDC9CAEECACBEFCBAF85
:103748000FAE0EAD0DAC0C120029E4FBFAF9F8121D
:1037580002C4709FAF0BAE0AAD09AC081203F08F1C
:103768000B8E0A8D098C08AF0BAE0AAD09AC081296
:103778002951AB0FAA0EA90DA80C12011E123CE686
:103788008F0F8E0E8D0D8C0CE51130E00B1203F0AF
:103798008F0F8E0E8D0D8C0CAF0FAE0EAD0DAC0CC9
:0137A80022FE
:1003A600E9D2E7C933E833F892D5EDD2E7CD33EC9D
:0703B60033FC5002B2D52216
:1003BD00EC30E7100FBF000C0EBE00080DBD0004A1
:1003CD000BEB6014A2D5EB13FCED92E7FD2274FF4D
:1003DD00FCFDFEFF22E480F8A2D574FF13FC7D80A6
:0303ED00E480EFBA
:1003F000ED33EC33600A047003BD8004ECB2E7FC1B
:0104000022D9
:103CAE0033DA929E35B16011377FE5FE3921848972
:103CBE003AAEC3FF3C1D955B3D6358473E75FDF024
:103CCE003F3172183F800000C2D50203E50203DBCC
:103CDE00BD80FA50F30203E2ED33EC330460F17B66
:103CEE003B7AAA79B8783F12011EED33EC3392D5A8
:103CFE00247B5011A2D570DB500BED448024045070
:103D0E0004A2D580CEEFFBEEFAEDF9ECF812036FBC
:103D1E00EFF582F404FC12033B12002DC082903C9E
:103D2E00AE7409120410ED33CC33D0F092D525F0D9
:0A3D3E00A2D57001C313CC13FD22BF
:10291D003E9248DA3ECCCCCD3F2AAAAB4000000017
:10292D003F8000003F9837F03FB504F33FD744FC9C
:10293D003E3172173EB172173F0515913EDE5BD9E0
:10294D00D2318002C231EDD2E7F8CD33EC330470D1
:10295D000BBD800592D50203E50203DB40FBD314CA
:10296D0060F2F5F07C3FEE7A00C39496C8948B40EC
:10297D00230AC89469C8941A401A0AC89468C8945E
:10298D001F40110AC8945AC89425400805F07A00D2
:10299D00CDC2E7CDC0F08C128D138E148F15EA23A6
:1029AD0023C0E0242DF582E43429F5831206B812F4
:1029BD00002DECC0E0EDC0E0EEC0E0EFC0E012068F
:1029CD009BA812A913AA14AB15120029D0E0FBD0B5
:1029DD00E0FAD0E0F9D0E0B2E7F81202278C128DC0
:1029ED00138E148F1590291D7403120401A812A9BA
:1029FD0013AA14AB1512011ED0E0600F2439F58215
:102A0D00E43429F5831206B812002D8C128D138E25
:102A1D00148F15D0E0C3947FFDE49400FC120336AF
:102A2D007B187A727931783F12011EA812A913AA68
:102A3D0014AB1512002D30310B7BD97A5B79DE7812
:052A4D003E12011E22F3
:10040100C0E0EFFBEEFAEDF9ECF812011ED0E0F5D9
:10041100F0EFFBEEFAEDF9ECF812069BA3A3A3A310
:10042100E8C0E0E9C0E0EAC0E0EBC0E0C0F01201E2
:100431001E1206B8A3A3A3A312002DD0F0D0E0FB97
:0D044100D0E0FAD0E0F9D0E0F8D5F0D422F8
:10044E00BB010689828A83E0225002E722BBFE02AC
:09045E00E32289828A83E49322DF
:10046700BB010CE58229F582E5833AF583E022504A
:1004770006E92582F8E622BBFE06E92582F8E22294
:0D048700E58229F582E5833AF583E49322AE
:10049400BB010689828A83F0225002F722BBFE0147
:0204A400F32241
:1004A600F8BB010DE58229F582E5833AF583E8F08C
:1004B600225006E92582C8F622BBFE05E92582C838
:0204C600F22220
:1004C800EF8DF0A4A8F0CF8CF0A428CE8DF0A42E48
:0204D800FE2202
:1004DA00BC000BBE0029EF8DF084FFADF022E4CC06
:1004EA00F875F008EF2FFFEE33FEEC33FCEE9DECCF
:1004FA00984005FCEE9DFE0FD5F0E9E4CEFD22ED15
:10050A00F8F5F0EE8420D21CFEADF075F008EF2F5E
:10051A00FFED33FD4007985006D5F0F222C398FD4F
:05052A000FD5F0EA22EC
:10052F00BB010A89828A83F0E5F0A3F0225006F717
:0F053F0009A7F01922BBFE06F3E5F009F3192214
:10054E00E88FF0A4CC8BF0A42CFCE98EF0A42CFC4C
:10055E008AF0EDA42CFCEA8EF0A4CDA8F08BF0A4CA
:10056E002DCC3825F0FDE98FF0A42CCD35F0FCEB29
:10057E008EF0A4FEA9F0EB8FF0A4CFC5F02ECD39EE
:0F058E00FEE43CFCEAA42DCE35F0FDE43CFC225B
:10059D0075F008758200EF2FFFEE33FECD33CDCC15
:1005AD0033CCC58233C5829BED9AEC99E582984098
:1005BD000CF582EE9BFEED9AFDEC99FC0FD5F0D675
:1005CD00E4CEFBE4CDFAE4CCF9A88222B800C1B99F
:1005DD000059BA002DEC8BF084CFCECDFCE5F0CBDD
:1005ED00F97818EF2FFFEE33FEED33FDEC33FCEB16
:1005FD0033FB10D703994004EB99FB0FD8E5E4F9D1
:10060D00FA227818EF2FFFEE33FEED33FDEC33FCBD
:10061D00C933C910D7059BE99A4007EC9BFCE99AB1
:10062D00F90FD8E0E4C9FAE4CCFB2275F010EF2FF6
:10063D00FFEE33FEED33FDCC33CCC833C810D707F6
:10064D009BEC9AE899400AED9BFDEC9AFCE899F831
:0E065D000FD5F0DAE4CDFBE4CCFAE4C8F922C4
:0E066B00C3E49FFFE49EFEE49DFDE49CFC22A0
:10067900EB9FF5F0EA9E42F0E99D42F0EC6480C8F8
:0606890064809845F02298
:0C068F00E6FC08E6FD08E6FE08E6FF2297
:10069B00E493FC740193FD740293FE740393FF22A5
:0D06AB00E6FB08E6F908E6FA08E6CBF822BF
:1006B800E493F8740193F9740293FA740393FB2298
:0C06C800ECF608EDF608EEF608EFF6225E
:1006D400D083D082E493F608740193F608740293ED
:0906E400F608740393F674047324
:1006ED00D083D082F8E4937012740193700DA3A39C
:1006FD0093F8740193F5828883E4737402936860B0
:06070D00EFA3A3A380DFAF
:104DFD00E4FFFE12044E600C0FEF70010E09E97016
:054E0D00F20A80EF2213
:104D2400E4FFFE800D6D60130FEF70010E09E97052
:0C4D3400010A12044E70EE7EFF7FFF2289
:00000001FF
